:020000040000FA
:08000000FF23831690002D2858
:08000800B700030EB8000C1054
:1000100005190D28301431100F28311430101C3000
:10002000B222AF002F1D28282F1C1C283008013AAF
:10003000B0003108013AB1000C30B222AC002C1CE7
:100040002828301C26288512051628280512851612
:10005000380E8300B70E370E09008501073099006E
:1000600083160F3085000C148312013090000B179B
:100070008B178501B401A201A301A401A501A6016A
:10008000A701A001A101051956280519582800301B
:100090002002031943280730200203185C28A10A14
:1000A0000C30210203195F28A00143280000000042
:1000B00000000000A00A4328A001A1014328A001DC
:1000C000A10105196F2805197128003020020319B4
:1000D00061280730200203187528A001612800005C
:1000E000000000000000A00A61288E018F01A0011D
:1000F000A101A11505198D2805198F2800302002AE
:1001000003197A280730200203189328A20D22141D
:10011000A10B8B289728A0017A280000000000007E
:100120000000A00A7A28A20D2210A10B8B28A001A2
:10013000A1010519A7280519A928003020020319D3
:100140009928073020020318AD28A0013B280000A1
:10015000000000000000A00A9928A001A101A1153B
:100160000519C3280519C528003020020319B02835
:10017000073020020318C928A30D2314A10BC1289E
:10018000CD28A001B0280000000000000000A00A57
:10019000B028A30D2310A10BC128A001A1010519AE
:1001A000DD280519DF28003020020319CF28073089
:1001B00020020318E328A0013B28000000000000F3
:1001C0000000A00ACF28A001A101A1150519F92856
:1001D0000519FB28003020020319E6280730200209
:1001E0000318FF28A40D2414A10BF7280329A0014C
:1001F000E6280000000000000000A00AE628A40D88
:100200002410A10BF728A001A10105191329051934
:100210001529003020020319052907302002031890
:100220001929A001A5290000000000000000A00A73
:100230000529A001A101A11505192F2905193129A9
:100240000030200203191C29073020020318352929
:10025000A50D2514A10B2D293929A0011C29000069
:10026000000000000000A00A1C29A50D2510A10B0C
:100270002D29A001A1010519492905194B29003093
:10028000200203193B290730200203184F29A0013F
:10029000A5290000000000000000A00A3B29A001E1
:1002A000A101A1150519652905196729003020024A
:1002B000031952290730200203186B29A60D2614B2
:1002C000A10B63296F29A001522900000000000042
:1002D0000000A00A5229A60D2610A10B6329A00137
:1002E000A10105197F290519812900302002031970
:1002F00071290730200203188529A001A5290000D3
:10030000000000000000A00A7129A001A101A115B0
:1003100005199B2905199D290030200203198829F8
:10032000073020020318A129A70D2714A10B992932
:10033000A529A00188290000000000000000A00AF3
:100340008829A70D2710A10B992922082306240626
:10035000250626062706031D3B282209031DB22970
:10036000B4013B28220803199B2AA21BC729703914
:10037000703A0319562AB4011C30B222AF00AF1AEA
:100380003B280030B2222206031D3B28E129B4019C
:100390001C30B222AF00AF1E3B282208193E0318C2
:1003A0003B281030B2222206031D3B281130B22216
:1003B0002306031D3B282408A3002508A4002608C3
:1003C000A5002308E039B600203A03191F2A360891
:1003D000803A0319332A3608E03A0319492A3608C5
:1003E000003A03199B2A3608403A0319002A3608B6
:1003F000603A0319002A3608A03A0319452A3B2817
:100400001C30B222AF002F1C082A2308203AA30078
:10041000AF18172A231E142AA31E112A85160512A7
:10042000162A05168512162A051285122316A31AF6
:100430001C2A301431103B28311430103B283F3037
:100440002302031D3B281C30B222AF002F1C2B2A95
:100450002408FF3AA400A41B302A301431103B2892
:10046000311430103B281C30B222AF00AF1C3B28A7
:10047000231E422A311C3F2A851605123B280516E9
:1004800085123B28051285123B28A31E482A3B28CB
:100490003B28EC302302031D3B28073024060319B8
:1004A000BD2A2508B5002408A2223928341CBB29FE
:1004B000221D692AA2183B28221C862A5F2A2308AB
:1004C000B200B2030310B20D0310B20DB414D8225F
:1004D0003B28B41C3B28220803393207B3000730FD
:1004E00033060319B82AA21D7D2A2308B500330854
:1004F000A222B301B401D8223B283308B22223023E
:10050000031D3B28B301B401D8223B28B41C3B286F
:10051000A21D922A2308B5001C30A222B201B40108
:10052000D8223B281C30B2222302031D3B28B201F3
:10053000B401D8223B2822082306031D3B2834148B
:1005400085013B2883169B008312350883169A0089
:100550001C1555309D00AA309D009C149C18AE2A95
:100560008312080083169B001C141A0883120800CB
:1005700008302306031DD52AC12A08302506031D8D
:100580003B280330B5000030A2220130B5000C300A
:10059000A222C030B5001030A2228030B500113048
:1005A000A2220230B5001C30A222B2013410392838
:1005B000FF308500E822E822E822E822E822E8224B
:1005C0008501080000000230B900B90BE52A0800D7
:1005D0004730BA00E222EC2ABA0BEA2A00000800EF
:0C05E0003C30BB00E822BB0BF22A0800F4
:0405EC0000340034A3
:02400E00843FED
:104200000300000000000000FF0000001E001D0071
:104210000400000000000000010000000000000099
:10422000C00080000000000000000000000000004E
:10423000000000000000000002000000000000007C
:10424000000000000000000000000000000000006E
:10425000000000000000000000000000000000005E
:04426000000000005A
:00000001FF
